:100000005FC200000C94E22F78C2000076C20000AC
:1000100074C2000072C2000070C200006EC2000014
:100020006CC200006AC200000C94182E0C94002FC1
:100030000C94CD2D62C2000060C200005EC20000C0
:100040005CC200005AC2000058C2000056C2000044
:1000500054C200000C94F42D50C200004EC20000A7
:100060004CC200004AC2000048C2000046C2000064
:1000700044C2000042C2000040C200003EC2000074
:100080003CC200003AC2000038C2000036C2000084
:1000900034C2000032C2000030C200002EC2000094
:1000A0002CC200002AC2000028C20000050109027B
:1000B000A10185020901A1000509190129081500FE
:1000C0002501950875018102050109300931158165
:1000D000257F95027508810609381581257F9501D0
:1000E00075088106050C0A38021581257F95017572
:1000F000088106C0C005010980A101850319012AF4
:10010000B700150126B700950175108100C0050CD8
:100110000901A101850419012AA002150126A002E6
:10012000950175108100C00660FF0961A101096297
:10013000150026FF00952075088102096315002629
:10014000FF00952075089102C005010906A101056F
:100150000719E029E7150025019508750181029529
:1001600001750881010507190029FF150026FF0008
:100170009506750881000508190129051500250156
:10018000950575019102950175039101C00000006C
:10019000000000000000000000000000000000005F
:1001A000000000000000000000000000000000004F
:1001B000007E0F00D4FFFFFFC700000078000000A2
:1001C00000000000002A2B280000000000000000B2
:1001D000000000000000000029000000002C1E3478
:1001E00020212224342627252E362D3738271E1F7E
:1001F000202122232425263333362E37381F0405A9
:10020000060708090A0B0C0D0E0F10111213141516
:10021000161718191A1B1C1D2F3130232D350405F4
:10022000060708090A0B0C0D0E0F101112131415F6
:10023000161718191A1B1C1D2F3130354C09025B7B
:1002400000030100A0FA09040000010301010009F4
:100250002111010001224400070581030800010962
:100260000401000203000000092111010001222203
:100270000007058203200001070503032000010990
:100280000402000103000000092111010001227B8A
:10029000000705840320000112010002000000088D
:1002A000ABC239390100010203011C037600690069
:1002B00061006C003A0066003600340063003200D2
:1002C00062003300630000002403530065007000E7
:1002D0006900610020006F0066006600690063002D
:1002E00069006E0061006C0069007300000010037B
:1002F00074006100700069006F006B00690000000D
:10030000040309041A00090013000A00000004286D
:1003100015241621172207001D001B0006001900D6
:10032000050028002B002C00000000000D000F002D
:100330001C00180000000B00112208310C24123898
:100340000E0010003600370038002A00167C4C00E2
:1003500000000000FD377A585A000004E6D6B44683
:100360000200210116000000742FE5A3E0033D0008
:10037000FA5D003D8889A654750A36E182AEFA7AA4
:100380001AA6FCA2ED495F2BD164DB9630A72B4661
:10039000AB9EF559ECD5D368B65BFED1E16EC41BBC
:1003A000B984165D8036B64DD8E275B0473F264217
:1003B000BF32485B382F89635FFA234565B210D39B
:1003C00089BEB88D7D3AF5C551E4BC448FC3D137A1
:1003D00087CD6AD96714BB943F4E71EF1618790424
:1003E0009C26142EC8FBB588C632A871ACB8E78627
:1003F00019EFD740EB2C6E7E2526BBF66602B9B905
:100400001CD9A4F5E284AFA6C9E43028A9CA944D4A
:10041000224601D6C197E207B54F423E0F41796CA3
:10042000A890B5C43C4CED16E652F86F24D0375C6A
:10043000EAEDD61FB3C4C5A61DAF2795A751D0BB03
:10044000DD451827E73CE0A190296894C5476C601A
:10045000DAFC0973285609722951EB41ACCEDCE471
:10046000F0EEE0753A292012202A9E9EFF0000003F
:10047000D80B8D6930EB368900019602BE0600006C
:10048000F8378A8BB1C467FB020000000004595A98
:10049000504F52514A4D4B4E2A4C2F30B6B7ABAC51
:1004A000BBBCA9AABDBECFD0CDCEDBDCD9DA0D0E48
:1004B0000B0F1A0508050905071811130408120C7B
:1004C00011241FBECFEFDAE0DEBFCDBF11E0A0E008
:1004D000B1E0E2EEF4E602C005900D92A83DB1074E
:1004E000D9F724E0A8EDB1E001C01D92A63DB20706
:1004F000E1F70E94A1260C94F33182CD9C01FB010F
:100500009A9581159F4120F5832F8170B32FB2708A
:10051000AA27732F74706627532F5870442734FF0F
:100520000DC08295807FAB2B09F08062672B09F0AC
:100530008064452B09F0806809950895AB2B09F07C
:100540008260672B09F08460452BB1F38860F4CF9B
:1005500080E0F2CF0C9441310895982F92959F70CE
:1005600024E0911102C020E0982F892F869586956E
:10057000811511F02E5F982F892F8695820F08958F
:100580008093D20408958093D304089521E030E04D
:1005900001C0220F8A95EAF78091D304822BF3CF12
:1005A00021E030E0A90102C0440F551F8A95E2F70F
:1005B000CA0180959091D3048923E5CF292F9830E3
:1005C00090F5853080F590E035E0239F800D911DFA
:1005D0001124282F277041E001C0440F2A95EAF723
:1005E00023E0969587952A95E1F7FC01EE0FFF1F12
:1005F000E80FF91FE65FFC4F20E030E070E051911A
:10060000DF01CB01022E02C0969587950A94E2F78E
:10061000817081958527842385278E932F5F3F4F97
:100620002330310561F70895292F983078F585300A
:1006300068F590E035E0239F800D911D1124682F0F
:10064000677023E0969587952A95E1F7FC01EE0FF8
:10065000FF1FE80FF91FE65FFC4F40E050E080E02D
:10066000219130E0062E02C0369527950A94E2F7D4
:1006700021703327042E01C0220F0A94EAF7822B3F
:100680004F5F5F4F4330510559F7089580E008955B
:100690009091D30421E030E0F90101C0EE0F8A957A
:1006A000EAF7D90102C0AA0FBB1F6A95E2F7EA2B4D
:1006B00001C0220F4A95EAF7892F8E23E81303C061
:1006C000892F822B60CF2095822F8923FBCF8091A9
:1006D000B8029091B702981301C008958F5F877098
:1006E000FACF90911E048095892380931E04282FB1
:1006F0002770211110C0891771F09091D50492FFD5
:100700000AC08695869586954BDF10921E0410923E
:10071000200410921F04089590911B04982B90932D
:100720001B040895982F909580911B048923809332
:100730001B04089580911A04811531F010921A0457
:1007400010922204109221040895803E9105D9F15F
:10075000C8F48133910509F482C048F489329105C7
:1007600009F472C08A32910509F480C00895893372
:100770009105E9F082389105D1F08533910509F4AE
:100780005EC00895843E9105D9F148F4823E9105FA
:1007900039F1833E910549F181EE90E00895863E5E
:1007A0009105C9F1873E910509F43EC00895209155
:1007B000D4042370211164C02091D50423FF14C0F8
:1007C00089E290E008952091D40420FD45C0309145
:1007D000D50430FF09C024FD24C083EE90E00895C5
:1007E0002091D40422FDF7CF08952091D40422FD56
:1007F00044C03091D50430FD43C024FFF5CF11C073
:100800002091D50421FFF0CF8091D40484FD09C04C
:1008100087EE90E008952091D40423FFE5CF24FFD4
:10082000F7CF80E090E008952091D40423FD2BC001
:100830003091D50431FFE1CF84EE90E0089520910E
:10084000D40425FFD1CFBCCF2091D40425FD1EC0F8
:100850002091D50423FFC8CF89E390E0089520912B
:10086000D40426FFC1CF8AE290E008952091D404F9
:1008700026FFBACF81E390E0089582EE90E00895DC
:1008800080EE90E0089586EE90E0089585E390E094
:1008900008959091D40492FF10C041E0282F247154
:1008A000243009F040E031E0282F2871283009F089
:1008B00030E0431711F02CE0822793FF10C041E095
:1008C000282F2471243109F040E031E0282F2871CD
:1008D000283109F030E0431711F02CE082273091E5
:1008E000D50430FF10C051E0282F2171213009F0CC
:1008F00050E041E0282F2871283009F040E05417DB
:1009000011F029E0822731FF10C041E0282F21712A
:10091000213109F040E031E0282F2871283109F019
:1009200030E0431711F029E0822794FD877E089577
:100930001F93CF93DF9309DFEC01811522E5920726
:1009400008F052C0811540E5940708F0CDC0803E04
:10095000910520F58D3C910508F0A1C0883A9105DC
:1009600070F4853A910508F097C081309105B9F18E
:100970000497813A910598F1C0E0D0E030C0885AE0
:1009800091094B97C8F7C85AD0E0CC0FDD1FC45966
:10099000DE4F0990D881C02DD46421C0811550E468
:1009A0009507B0F4C11580E2D80708F0B3C0C83E7F
:1009B000D105A8F0CE019A9581159F41E8F68D2FBB
:1009C00068DF182FCE019927C0DEEC01D12B07C0BC
:1009D0009927BBDECC27DF70C82BD92BD06ACE017C
:1009E000DF91CF911F910895803842E59407C8F5B3
:1009F000803652E5950708F05BC0C03482E5D80721
:100A0000D0F4C03292E5D90708F04BC08C2F869500
:100A1000869520E2829FC0011124C37021E030E05E
:100A2000A90102C0440F551FCA95E2F7EA01C82B7D
:100A3000D92BDD68D4CF8C2F86958695877050E2B0
:100A4000859FC0011124C37021E030E0A90102C0DC
:100A5000440F551FCA95E2F7EA01C82BD92BDC6871
:100A6000BECF803C52E5950758F48F71C03AD2450D
:100A7000A0F590E0982F8827EC01C46FD06AAFCF23
:100A8000805C9245809708F077CFDC2FCC27CC276D
:100A9000DF71C06FD06AA3CFA497D064A0CFD06518
:100AA0009ECFCF71D0E0DC2FCC27C16FD06A97CF1B
:100AB00086958695877020E2829FC0011124C370BD
:100AC00021E030E0A90102C0440F551FCA95E2F7AA
:100AD000EA01C82BD92BDA6882CFDBDEC82FD0E041
:100AE000DC2FCC27D0627BCF8F71D3DE93E0CC0F8D
:100AF000DD1F9A95E1F7CC27DF70282F30E084FFC7
:100B000005C050E1859F900111243327C22BD32BC0
:100B1000D06965CF8D2F8F71BCDE182FCE0199273C
:100B200014DEEC01D12BDECF80E0089581152CE797
:100B3000920741F42091890230918A02232B11F40B
:100B400080E090E00895E0E9F3E080E090E06FE578
:100B500075E242E855E224EF35E2778366835187F8
:100B600040873387228797878687019670968830DB
:100B7000910599F70895FB01811520E2920728F469
:100B8000811541E0940738F408959C0130522115F5
:100B9000304348F00895392F94FF02C03295307FDA
:100BA0002081232B208399270895462B22FF0FC0F5
:100BB000982F92959F708F70892B962F92959F708A
:100BC0006F70692B942F92959F704F70492B982FBF
:100BD0009623961309C050E04095509590E0482325
:100BE000592381E0452B09F080E0089510926404B8
:100BF00010926304E3E2F4E08581811102C0148263
:100C00001682379684E0EB35F807B1F70895AC010A
:100C10003091660460916504232F621301C008952A
:100C2000822F90E0FC01EE0FFF1FE55AFB4F019071
:100C3000F081E02DE417F50791F467E0649FF0017F
:100C4000659FF00D1124ED5DFB4F41E044832313BC
:100C5000E6CF0196837099278093660408950196E4
:100C6000282F2370DACF0F931F93CF9301E010E06A
:100C7000082E01C0000F0A94EAF7C09119049C2FB6
:100C80009023911115C090911E0496959695969576
:100C9000891306C010921E041092200410921F04A3
:100CA00075DCC027C0931904CF911F910F9108954F
:100CB00077DCF7CF282F35EB2303C001112497FFF2
:100CC00004C080589109892F089580589F4FFBCF09
:100CD00080911B0380FD14C081FD14C082FD16C0ED
:100CE00080911A03811581F08E3180F420E5829F76
:100CF000C00111246EE170E00E942831862F089512
:100D000084E1089588E2089588E0089580E50895D3
:100D100080911B0380FD17C081FD17C082FD19C0A3
:100D200080911903811599F0883298F428E0829F08
:100D3000C001112468E270E00E942831611571053C
:100D400051F0862F089562E0FCCF64E0FACF61E0B5
:100D5000F8CF68E0F6CF81E008959091770389029B
:100D60009001112437FF03C08093770308952F3734
:100D700031051CF4980F9093770308959C0180E04F
:100D800090E0F901E80FF91FE491E41307C091E046
:100D90008927F901E80FF11D8491089501968617BE
:100DA00080F380E00895FA01309709F009950895DD
:100DB0008091A102811569F0E091AD02F091AE023F
:100DC000309739F00190F081E02D309711F00995BE
:100DD000089580E00895A3E0B0E0E1EFF6E00C9420
:100DE00001319C01809108029091090282179307BA
:100DF000B1F03093090220930802E091AD02F09126
:100E0000AE02309761F00084F185E02D309739F023
:100E100083E089833B832A83CE010196099523963B
:100E2000E2E00C941D31A3E0B0E0E9E1F7E00C94BE
:100E300001319C018091060290910702821793076D
:100E4000B1F03093070220930602E091AD02F091D9
:100E5000AE02309761F00084F185E02D309739F0D3
:100E600084E089833B832A83CE01019609952396EA
:100E7000E2E00C941D319C01FC0132968FEF90E072
:100E80004191461751F08F3F19F4411101C0892F4C
:100E90009F5F9630A9F78F3F09F40895280F311D01
:100EA00087FD3A95F901628308959C01FC01329611
:100EB000285F3F4F8191861302C0DF011E92E21727
:100EC000F307C1F708958091010108952FB7F894B1
:100ED0008091020290910302A0910402B091050258
:100EE0002FBF0895962F2091D50422FF0EC0682FA2
:100EF000660F660F660F692B60931E0447DBE6DF03
:100F00009093200480931F04089540CB90911A047D
:100F1000292F2823211559F08095892380931A04BD
:100F2000811531F0D3DF809321049093220408953A
:100F300080E090E0F8CFCADF20911E0330911F03BC
:100F4000232B211521F080937A0290937B0220912C
:100F5000200330912103232B211521F08093780267
:100F600090937902E091AD02F091AE02309759F082
:100F70000680F781E02D309731F082E080931C03EA
:100F80008CE193E009950895611509F441C0E3E30C
:100F9000E80FE33148F4F0E0EB50FE4C0C943B31A9
:100FA00097DE819580931F03C6CF92DEFBCF90DE44
:100FB000819580931E03F8CF8BDEFBCFA9DE809353
:100FC0002003F2CFA5DE8195FACFA2DE8195809332
:100FD0002103EACF9DDEFBCF815D990B21E030E05C
:100FE00001C0220F8A95EAF780911D03822B80931E
:100FF0001D03DACF80911B03816080931B03D4CF44
:1010000080911B038260F9CF80911B038460F5CF30
:1010100040911E038D3C59F480911F0387FF0DC042
:1010200010921F03411559F410921A0308C08E3C08
:1010300081F480911F0318169CF3411581F0809173
:10104000200390912103892B8111AECF10921903B7
:10105000ABCF8F3C41F447FFF0CF10921E0380913D
:101060001F038115E0CF803D19F41416B4F3E5CFCA
:1010700090912003893D29F41916FCF61092200363
:10108000DCCF8A3D19F497FFD8CFF8CF9091210398
:101090008B3D29F497FFD1CF10922103CECF8C3D09
:1010A00019F41916CCF3C9CF9FE2980F983090F439
:1010B000815D990B21E030E0B90102C0660F771F16
:1010C0008A95E2F7CB01809590911D038923809347
:1010D0001D03B3CF8D3D31F480911B038E7F809330
:1010E0001B03ABCF8E3D21F480911B038D7FF7CF87
:1010F0008F3D09F0A2CF80911B038B7FF0CF2FB7DC
:10110000F894609102027091030280910402909120
:1011100005022FBF08950F931F938091A10281159F
:1011200021F0EDDF1F910F910895E9DF0091A302F7
:101130001091A4022091A5023091A602600F711FA8
:10114000821F931FEFCF87E797E790930108809363
:10115000000888E19AE00FB6F894A89580936000A3
:101160000FBE90936000FFCF0895FC019B0180911A
:10117000F8019091F9018617970740F0672B29F441
:101180008091E8008E778093E800C90140E00097E5
:1011900041F4411106C08091E80082FF2FC080E039
:1011A000089520918B022115A9F12530A9F12091F4
:1011B000E80023FD2DC02091E80022FDECCF209116
:1011C000E80020FFE4CF3091F3002091F200009777
:1011D00019F02830310558F041E02830310509F088
:1011E00040E02091E8002E772093E800D0CF419195
:1011F0004093F10001972F5F3F4FE9CF80918B0221
:10120000811541F0853041F08091E80083FFC3CF24
:1012100081E0089582E0089583E008958091F201CD
:1012200087FF13C08091E80082FF06C08091E8002C
:101230008B778093E800089580918B028111F2CF23
:10124000089580918B028115D9F38091E80080FF89
:10125000F8CF8091E8008E77ECCF2091E4003091B8
:10126000E50095E6A9012091EC00822F817020FF16
:1012700006C08091E80080FF06C080E008952091BC
:10128000E80022FD1AC080918B02811589F085301B
:1012900089F08091EB0085FD0FC02091E400309132
:1012A000E50042175307F9F29A95E1F684E00895B4
:1012B00082E0089583E0089581E00895E8EDF0E08C
:1012C00080818E7F80831092E2001092DA0010926B
:1012D000E100A0EEB0E08C9181608C9380818F77EB
:1012E000808319BCA7EDB0E08C918E7F8C938081B8
:1012F0008F7E80831092F1010895E091AD02F0910C
:10130000AE02309739F00284F385E02D309711F06A
:1013100060E209950895FC01AC014C5F5F4F8FEFCF
:1013200061E39191892728E030E0982F990F87FF9A
:1013300009C0892F862721503040B9F7E417F507F7
:1013400081F70895892FF7CF982F9093E900891797
:1013500071F07091EC002091ED005091F00021FDB2
:1013600009C09F5F973089F78093E9000895762F31
:10137000242F50E03091EB003E7F3093EB00309112
:10138000ED003D7F3093ED003091EB003160309304
:10139000EB007093EC002093ED005093F00020914F
:1013A000EE0027FDDECF0895A0E0B0E0EAEDF9E021
:1013B0000C94FB30C8EDD0E088818F7E8883E7ED08
:1013C000F0E080818160808384E082BF81E080934F
:1013D000F10188818E7F888302EE10E0F80110828F
:1013E0001092DA0081EEC82ED12CF601108288818D
:1013F0008F77888388818068888388818F7D8883C0
:1014000019BC10928B021092F00110926E02109291
:10141000EF0190EEE92EF12CF70180818B7F808324
:1014200088818160888342E060E080E08DDFF601A2
:1014300080818E7F8083F8018081816080838081BC
:1014400088608083F70180818E7F808388818061BE
:101450008883CDB7DEB7E8E00C941731E091B8028D
:101460009091B70229E0E91302C080E00895AE2F01
:10147000B0E02E9FF0011124E754FD4F3181361367
:1014800006C03081381303C03581341304C0FD0118
:101490003196E770E8CF81E008950F931F93CF93C3
:1014A000DF938B01EA0190918B02943051F5809388
:1014B000E9008FEF9091E80095FD06C095ED9A95B3
:1014C000F1F700008A95B1F78091E80085FF19C017
:1014D000C4DE811111C08091E80085FD06C08091B5
:1014E000E8008E778093E800F3CFF80181918F01B7
:1014F0008093F100219779F78091E8008E778093AF
:10150000E800DF91CF911F910F910895792F6032FC
:1015100029F440E250E0682F82E0BFCF0895CF93D6
:10152000DF93D82FC92F48E050E0682F792F81E052
:10153000B4DF88E0ED2FFC2FAAEFB1E001900D920F
:101540008A95E1F7DF91CF910895BC0146E050E024
:1015500084E0A3CFBC0143E050E084E09ECFA0E054
:10156000B0E0E5EBFAE00C94F930F82EE92EB62E57
:10157000A72E8A018091EC019AE0C92ED12C8A30E5
:1015800018F0CC24C394D12CC1E0D0E06B2D7A2D7F
:101590008F2D9E2DF8010995811116C02196CC162C
:1015A000DD0694F0CC9FC001CD9F900D900D1124CD
:1015B00020E030E045E34A95F1F700002F5F3F4F10
:1015C00028173907B9F7E2CFCDB7DEB7EAE00C94B8
:1015D00015319091D50492FB222720F9281771F03C
:1015E00080FB92F99093D5046091D4047091D50456
:1015F00084E090E00E94D83182E073C80895609141
:1016000016048CE090E00C94BE311F93CF93DF93CF
:10161000962F122F632F282F292B2830C8F44530FE
:10162000B8F4C42FD0E0CC0FDD1F2AE0929FC00D8C
:10163000D11D112490E5899FC00DD11D1124CE012B
:1016400089960E94BE31612FCE018A960E94BE31DA
:10165000DF91CF911F910895CF93DF93C0911B0429
:1016600080911D04C82B80911A048115E1F02EDCB5
:101670002091210430912204821B930B88389341DE
:1016800008F058D8D0911A0420E08CED91E0FC01CC
:101690003081019631112F5F31E0823E9307B9F717
:1016A000211148D8CD2BC093DA0148E050E06FEA11
:1016B00072E08AED91E00E947531892BB9F088E0E3
:1016C000EAEDF1E0AFEAB2E001900D928A95E1F720
:1016D000E091AD02F091AE02309741F00280F381CB
:1016E000E02D309719F08AED91E00995DF91CF91C7
:1016F0000895CF9310921B04C6E0ECEDF1E0DF01FA
:101700008C2F1D928A95E9F780E090E064DB80E001
:1017100090E089DB10921D049FDFECE1F3E0DF0134
:101720001D92CA95E9F710921A03109219031092AC
:101730001B0301DCCF910895DCDF2FEF84E39CE0F5
:10174000215080409040E1F700C0000088E19AE01D
:101750000FB6F894A895809360000FBE9093600038
:10176000FFCFAAE2B0E0E7EBFBE00C94003182EFA0
:1017700091E0FC0101962091F100208321E08A3F55
:101780009207B9F78091F301893009F457C0C8F482
:10179000823009F4B2C0833009F482C0813081F113
:1017A0008091E80083FFE6C08091F2019091F301FF
:1017B0009A3008F0DFC0E92FF0E0E85FFD4C0C94B0
:1017C0003B318A3009F489C08B3051F78091F201A6
:1017D000813231F78091F6019091F701892B01F761
:1017E0008091E800877F8093E80018DD81E0909188
:1017F000F401911101C080E0809302017ADFD0CF23
:101800008091F201813A61F68091E800877F8093B0
:10181000E8008091F6019091F701892B59F060E082
:1018200080E090E070E0A1DC8091E8008B7780930D
:10183000E800B6CF68E08AEF91E0F4CF8091F20142
:10184000813209F0ADCF8091F6019091F7018D7F43
:10185000892B09F0A5CF8091E800877F8093E8006D
:101860008091E80082FF17C09091F3008091F20010
:10187000029731F48091F100813011F0863021F42B
:101880008091F100809301018091E8008B77809333
:10189000E800C4DC85CF80918B028111E1CF80CF3D
:1018A0008091F201813A09F07BCF8091F60190910D
:1018B000F701892B09F074CF8091E800877F80932E
:1018C000E8008091E80080FFFCCF809102018093C6
:1018D000F1008091E8008E77DACF8091F2018132B9
:1018E00009F05ECF8091E800877F8093E80096DC66
:1018F0008091F5018093000153CF8091F201813AEC
:1019000009F04ECF8091E800877F8093E8008091B6
:10191000E80080FFFCCF80910001D9CF803889F0AA
:10192000823841F58091F6018F70873018F58093E9
:10193000E9008091EB0085FB882780F91092E9008F
:1019400006C080916E02880F9091EF01892B9091D3
:10195000E800977F9093E8008093F1001092F100E7
:101960008091E8008E7723C0811116C08091F40128
:10197000813009F18091E80083FF0AC08091E8007E
:10198000877F8093E8008091EB0080628093EB007A
:10199000AA96E3E00C941C31823061F78091F40147
:1019A000811581F01092E9008091E800877F809393
:1019B000E80034DCDFCF81E0933009F080E08093F1
:1019C0006E02F0CF8091F6018F702FEF280F263036
:1019D00088F68093E9002091EB0020FFE3CF93305D
:1019E00031F48091EB0080628093EB00DBCF90912B
:1019F000EB0090619093EB0021E030E0A90102C080
:101A0000440F551F8A95E2F74093EA001092EA00CE
:101A10008091EB008860E8CF8111ACCF1091F40188
:101A20001F778091E3008078812B8093E300809181
:101A3000E800877F8093E800F1DB8091E80080FF79
:101A4000FCCF8091E30080688093E30083E0111174
:101A500001C082E080938B028DCF8058823008F0E5
:101A600089CF8091F4019091F5018C3D53E0950769
:101A700091F583E08A838AE289834FB7F894DE0187
:101A8000139620E03EE051E2E32FF0E05093570040
:101A9000849120FF03C082958F703F5F8F708A30E2
:101AA000C0F0895C90E08D939D932F5F243161F7A6
:101AB0004FBF8091E800877F8093E8006AE270E082
:101AC000CE01019652DB8091E8008B778093E8008D
:101AD00051CF805DE7CF292F33272330310509F41B
:101AE0004EC078F52130310509F488C08BE590E0CF
:101AF000EDE3F2E02230310509F03CCF2091E8001F
:101B0000277F2093E8002091F8013091F901821796
:101B1000930708F49C0140E02115310509F073C0DA
:101B2000411171C08091E80082FDCDCF80918B0280
:101B3000811549F2853039F28091E80083FFF2CFB8
:101B4000C2CF8091F6019091F7012132310509F45D
:101B500046C02232310509F00DCF8330910508F0DF
:101B600009CFFC01EE0FFF1FE25AFE4F0190F081FA
:101B7000E02D855A9E4FDC018C9190E010C09C01B5
:101B80003327823021F12330310568F4232BB9F457
:101B9000E0E0F3E0E4918E2F90E0E0E0F3E00097E6
:101BA00009F4E8CEABCF2330310509F0E3CEEAEA01
:101BB000F2E0E4918E2F90E0EAEAF2E0F0CFEEEE70
:101BC000F2E0E4918E2F90E0EEEEF2E0E8CFE8EC68
:101BD000F2E0E4918E2F90E0E8ECF2E0E0CF833089
:101BE000910508F0C7CEFC01EE0FFF1FEC59FE4F28
:101BF0000190F081E02D89E090E080CF82E190E0DB
:101C0000E8E9F2E07BCF80918B02811509F45BCF8C
:101C1000853009F458CF8091E80083FD54CF80913E
:101C2000E80082FD7FCF8091E80080FF75CF909122
:101C3000F3008091F2002115310519F088309105EB
:101C400050F041E0089709F040E08091E8008E777D
:101C50008093E80061CF44914093F1003196215088
:101C600031090196E8CF803809F084CE8091E800F0
:101C7000877F8093E8008091F0018093F10070CE1F
:101C8000811178CE1091F401123008F073CE80915A
:101C9000E800877F8093E8001093F001BFDA111508
:101CA000D9F084E080938B0242E061EC81E04CDB70
:101CB00042E261EC84E048DB42E261EC82E044DB3A
:101CC00042E260EC83E040DB80918B02843051F48F
:101CD00082E0809303014ECE8091E30087FDE1CF47
:101CE00081E0E0CF81E0F5CFCF93C82F811599F047
:101CF0008CEF8C0F813A88F4ECEDF1E082EE91E00C
:101D00002191C217B1F18E179F07D1F76C2F8AED81
:101D100091E0B1D8A1DCCF91089580E28C0F88309A
:101D200048F4C77081E001C0880FCA95EAF70E94A5
:101D30008C03F0CF8BE58C0F833030F42C2F2452A2
:101D4000330BC90148D8E7CFE8E5EC0FEB3148F495
:101D5000F0E0EE0FFF1FEE55FE4F8081918163D8BA
:101D6000DACF83E38C0F8331B0F661E08C2F0CD98E
:101D7000D2CF6C2F8AED91E098D86EDCC7CFCF938D
:101D8000DF93EC01805E9109089720F064E170E137
:101D9000209711F468E070E1CE010E947E028C2F42
:101DA000A3DFDF91CF910895811561F19CEF980F2A
:101DB000913A28F4682F8AED91E077D84DCC90E2E3
:101DC000980F983050F4877091E001C0990F8A9570
:101DD000EAF7892F0E949203F1CF9BE5980F933089
:101DE00020F480E090E00C94EB0698E5980F9B318E
:101DF00018F480E090E017C893E3980F933110F443
:101E000060E0C2C80895CF93DF93EC01CDDFCE012F
:101E1000805E9109089720F06DE170E1209711F440
:101E20006EE070E1CE010E947E02DF91CF910895B5
:101E30000F931F93CF93DF938C01EB01A0DF2097CB
:101E400039F4C801E0DFDF91CF911F910F91089520
:101E50008FE99FE00197F1F700C000002197EFCFD5
:101E60001F93CF93DF93182FEB013EDF209731F4C0
:101E7000812F9ADFDF91CF911F9108958FE99FE025
:101E80000197F1F700C000002197F0CF60E570E006
:101E9000893311F060E070E0E3CFA0E0B0E0E3E56B
:101EA000FFE00C94FC30E82FF0E0E354FE4FD490B8
:101EB000282F26952695269530E0F901E355FE4F0B
:101EC0000491877010E0082E02C0159507950A94BA
:101ED000E2F701701127F901E356FE4FE490F12C6F
:101EE000082E02C0F594E7940A94E2F7E0FAEE2493
:101EF000FF24E0F8F901E357FE4FC491D0E002C09F
:101F0000D595C7958A95E2F7C170DD2701151105B2
:101F100011F081EEE9DEE114F10411F086EEE4DE69
:101F200060E070E08D2D9CDFE114F10411F086EE8D
:101F30003BDF0115110511F081EE36DFCD2B11F0DD
:101F40008CE2A4DFCDB7DEB7E7E00C9418319091B6
:101F50001604923061F48A3040F4875F90E06AE0C2
:101F600070E00E942831875A91CF8650FDCF96EFBE
:101F7000980F963010F0805D90CF895AFDCFCF93A7
:101F8000DF93EC0188818115D9F0813009F03DC0E3
:101F90008981813021F48A81239678DFF3CF8230E2
:101FA00021F48A812396A0DEEDCF833021F48A814B
:101FB0002396FADEE7CF843031F022968111E2CF0A
:101FC000DF91CF9108958A81239620E030E09AE056
:101FD000682F6053770BAB016A30710560F02115F3
:101FE000310561F3EFE9FFE03197F1F700C0000040
:101FF00021503109F4CF929FB001939F700D1124AD
:102000009A01260F371F8991E3CF219646DFBACF79
:10201000811519F00E948C031FCB0895811519F0CA
:102020000E94920319CB0895811531F090911D04FF
:10203000892B80931D0410CB0895811539F080956C
:1020400090911D04892380931D0406CB08958091EF
:102050008C03811521F082E2F0DF10928C03089549
:10206000CF93DF93EC014A855B856E857F850E9467
:10207000D3069B81909580911D04892380931D0434
:102080008C810E949203E8DA86E0FE0111928A9523
:10209000E9F7DF91CF910895CF93DF93EC018D8124
:1020A00081FD13C082608D8380911D049B81892BEB
:1020B00080931D048C810E948C03CEDA488559855B
:1020C0006E857F85CE010E94D30610921104109276
:1020D00010048D8180FD02C0CE01C2DFDF91CF915F
:1020E0000895ACE0B0E0E7E7F0E10C94FB30FE01CE
:1020F000319688E0DF011D928A95E9F744E051E0CE
:10210000BE016B5F7F4F8F016A01EE24E394F12CD7
:1021100030E0D6012D916D012F3F81F0822F829505
:102120008F70805E90E0DC018C9190E02F7002C097
:10213000959587952A95E2F780FF68C080E0F82A98
:102140003F5FEE0C353029F7F1924B5F5F4FE6179A
:10215000F707D1F648E050E0B80183E692E00E942C
:1021600075319C01892B41F088E0F801A3E6B2E0CB
:1021700001900D928A95E1F700916C0210E00F57E3
:102180001D4F232B09F444C081E08093EB010E9492
:1021900066079093EA018093E9018091A10281157D
:1021A00009F491C07E01B9E0EB0EF11C84E0F70167
:1021B00011928A95E9F78091EC018A3008F04CC0C1
:1021C0004DEF51E1B701C801CAD9811509F469C0C1
:1021D00042EA51E1B701C801C2D9811509F461C0D1
:1021E0001092EC0180916B0290E044E050E0B70166
:1021F0008F579D4F0E94753121E02093E801892B74
:1022000009F041C02C96E8E00C9417318E2D97CF41
:102210008091EB01811509F4C0CFE090E901F090C5
:10222000EA010E9466078E199F09059708F4B5CF49
:1022300044E050E063E672E0C8010E947531892BEA
:1022400041F084E0E3E6F2E0D80101900D928A9536
:10225000E1F71092EB01A1CFC090E601D090E70129
:102260000E9466078C199D09843F914008F0A8CF11
:102270008091E801811531F284E0D7011D928A95A1
:10228000E9F71092E801E0916B02F0E0EF57FD4FA3
:1022900089859A85AB85BC8580839183A283B3832E
:1022A000B1CF8091EC018F3F39F40E946607909383
:1022B000E7018093E601DCCF8F5F8093EC018A30E9
:1022C00008F490CFF2CFF80180819181A281B3818F
:1022D0008093910290939202A0939302B093940200
:1022E00081E992E018D880939002C0909502D09036
:1022F0009602E0909702F09098028091E20190910E
:10230000E301A091E401B091E501C816D906EA06FF
:10231000FB0609F477CFC092E201D092E301E0928C
:10232000E401F092E5010E947F08C61AD70AE80A84
:10233000F90AC092A302D092A402E092A502F09200
:10234000A60260CFCF92DF92EF92FF921F93CF93BE
:10235000DF9300D000D0CDB7DEB7C0908C02D09014
:102360008D02E0908E02F0908F020E947F086C191F
:102370007D098E099F0911E064367105810591057B
:1023800078F10E948B08DC01CB010296A11DB11DE2
:1023900089839A83AB83BC83809136019091370106
:1023A00080579D4F20913501422F50E0253010F08D
:1023B00044E050E0BE016F5F7F4F0E94823182E0B7
:1023C00090E00E948330182F811551F00E947F0801
:1023D00060938C0270938D0280938E0290938F0293
:1023E000812F0F900F900F900F90DF91CF911F9141
:1023F000FF90EF90DF90CF9008958F929F92AF92D1
:10240000BF92EF92FF921F93CF93DF9300D000D043
:102410000F92CDB7DEB77B0180E090E00E94833061
:10242000182F811509F464C080912801482F50E0CD
:10243000811511F041E050E06091290170912A016D
:1024400060577D4FCE0105960E94823180909D029B
:1024500090909E02A0909F02B090A0020E947F08E0
:10246000681979098A099B09643671058105910506
:1024700038F481E992E00E948B099D818917C1F1AE
:1024800081E090E00E948330811509F43FC0809183
:102490003001482F50E0853010F044E050E060916A
:1024A00031017091320160577D4FCE0101960E943B
:1024B000823181E992E00E948B099D81891326C0B7
:1024C0000E947F0860939D0270939E0280939F02FA
:1024D0009093A00289819A81AB81BC8180939902FB
:1024E00090939A02A0939B02B0939C0281E00FC04C
:1024F0008091910290919202A0919302B0919402E6
:1025000089839A83AB83BC831111E4CF80E040912F
:10251000990250919A0260919B0270919C02F7017E
:1025200040835183628373830F900F900F900F90BD
:102530000F90DF91CF911F91FF90EF90BF90AF90E0
:102540009F908F9008950F931F93CF93DF93982FB1
:10255000962B983020F5453010F5C42FD0E0CC0FE5
:10256000DD1F2AE0629FC00DD11D112430E5839F3D
:10257000C00DD11D1124CE0189960E94A231082FD1
:1025800010E0102F0027CE018A960E94A2319801F8
:10259000282BC901DF91CF911F910F91089580E001
:1025A00090E0F8CF462F672F2091A9023091AA0220
:1025B000232B81F4703F39F4403F61F48091A702EE
:1025C0009091A8020895982F972B983018F44530D1
:1025D00008F4B9CF80E090E00895A0E0B0E0E3EF28
:1025E000F2E10C94FC307C010091D3048091D20480
:1025F000082BC7E0D0E010E0C8010C2E02C0959572
:1026000087950A94E2F780FD09C02197A8F7D12C9D
:102610008D2DCDB7DEB7E7E00C941831DC2EB70175
:102620008C2FC0DF0E949804019779F3F1CF0F93AC
:102630001F93CF93FC0187819085009789F4858152
:1026400000811181811581F0611571F0C801C5DF2C
:10265000C82F682FC8010E94DE02B8018C2FA2DFAC
:10266000CF911F910F910895C8010E941403C82FA4
:10267000F4CFCF93DF93D82FC92FAFDF6D2F7C2FEF
:1026800091DF0E949804DF91CF910895FC0184812D
:102690008115B1F0878190850097A1F00E94980480
:1026A000282F92959F709630B9F080F4925F9F70BA
:1026B000923030F4203FD1F058F481E0283E58F0B9
:1026C00080E0089580819181D4DFEACF9A5FEFCFD7
:1026D00081E0243FA9F7089591E0813F09F090E05F
:1026E00081E0283E08F080E0892B089581E008957C
:1026F000382F292FCB01A32FB22F87389105A105A1
:10270000B10520F487589C4F0C94A23180E00895C5
:1027100085E290E00E94A2318D3B89F486E290E050
:102720000E94A2318C3159F487E290E00E94A231DC
:1027300091E0843F09F090E0892F8170089580E056
:10274000FCCFAAE0B0E0E7EAF3E10C94F730C090E8
:102750008902D0908A0281E090E090938A0280936F
:10276000890210E084E0A82E83E0B82E00E01AC0B1
:1027700021E030E0111104C0F401859195919C0194
:102780004F2D602F812F0E94050BF39482E0880E5D
:10279000911C95E0F912ECCF0F5FEAE0AE0EB11C90
:1027A000083019F04501F12CE3CF1F5F1830D1F646
:1027B0001A8219821C821B821E821D8218861F8229
:1027C00088EC90E09A87898709EA12E0CE010196A9
:1027D0007C014AE050E0B801C7010E94DC31065F8D
:1027E0001F4F093F92E01907A1F78AE0F701119204
:1027F0008A95E9F74AE050E0B801C7010E94DC3150
:10280000065F1F4F0934F3E01F07A1F786E0F701C9
:1028100011928A95E9F746E050E0B801C7010E949D
:10282000DC310A5F1F4F0937F3E01F07A1F7D09291
:102830008A02C09289022A96ECE00C941331AAE035
:10284000B0E0E5E2F4E10C94FB30EBE0F2E080E58F
:10285000DF011D928A95E9F7E3E2F4E088E3DF0106
:102860001D928A95E9F78BE0C82E82E0D82E7F0171
:1028700009EF12E0F701D182C0824AE050E0B801CE
:10288000CE0101960E94923188E0FE013196D60178
:1028900001900D928A95E1F789859A85D701139663
:1028A0009C938E931297BAE0CB0ED11CE7E0EE0E0C
:1028B000F11C065F1F4F0934F3E01F07D9F62A9673
:1028C000E8E00C941731A6E0B0E0E9E6F4E10C94FE
:1028D000FC300CE213E089E4E82E83E0F82E98E067
:1028E000D92E46E050E0B701CE0101960E94923108
:1028F000F8018D2D11928A95E9F7B8016C5F7F4F31
:1029000089819A810E94BB05F80191838083B80177
:102910006B5F7F4F8B819C810E94BB05F801938385
:1029200082838D8186838E818783F6E0EF0EF11C92
:10293000085F1F4F89E7E81683E0F80691F62696B0
:10294000E7E00C941831282FCB01283070F44AE0CE
:10295000249F90011124B90167557D4F4AE050E052
:102960000E94923180E090E008958FEF9FEF0895EC
:10297000AAE0B0E0EEEBF4E10C9401319C01975534
:102980008115914068F4BE016F5F7F4F822FDBDFBE
:10299000892B31F489859A852A96E2E00C941D31C1
:1029A00088EC90E0F9CFA0E0B0E0E9EDF4E10C9420
:1029B000FC30162FD72FC42FD22E8115A1F04093B3
:1029C00017040E9466079093EE018093ED01C77093
:1029D00081E001C0880FCA95EAF71ADBCDB7DEB7F0
:1029E000E7E00C94183190911704491333C0E0903C
:1029F000ED01F090EE010E9466079C012E193F093F
:102A00007901812F9D2FB4DFE816F90618F5D0E281
:102A1000DD0DCD1591F0C77011E0812F01C0880F39
:102A2000CA95EAF7FBDAD83040F48D2D877001C0E3
:102A3000110F8A95EAF7812FEBDA802F27DAD83049
:102A400068F62D2D277081E001C0880F2A95EAF7DE
:102A5000E5DAC4CFC77081E001C0880FCA95EAF7F4
:102A6000F7CFAAE0B0E0E7E3F5E10C94F1307C01A8
:102A7000DC0114968C91811509F448C161E0C7010D
:102A8000D6DD8C01F7018581811521F1809110043B
:102A9000909111040097F1F008171907D9F0FC0183
:102AA000FF27887F9927892B09F04BC084E0EE0F20
:102AB000FF1F8A95E1F7E057FC4F8581846085838D
:102AC00011830083CF01E8DA10921D0461E0C70191
:102AD000AEDD8C018091810381113AC0D70115963A
:102AE0008C91811509F4C9C00115B0E51B0708F0E8
:102AF000AFC00115E0E21E0708F00CC10115F7E0B8
:102B00001F0731F108F5C801805E9109089700F1AF
:102B100030911B0480911D0420911A0499E0F70163
:102B2000ADE6B3E001900D929A95E1F7109375032D
:102B30000093740310927703832B822B80936C0392
:102B400007C0E0E0F0E0B9CF01153FE0130701F75F
:102B5000F70185818111DBC1011527E5120708F412
:102B6000E6C2011538E5130710F00C943B1F68010D
:102B700047E5D41A62E873E08C2DE5DE892B31F548
:102B8000C601F4E0880F991FFA95E1F7FC01E057C0
:102B9000FC4F2281213009F09AC2209182033091AA
:102BA0008303232B99F02091840330918503232BF9
:102BB00069F02091860330918703409188035091FA
:102BC0008903242B352B232B09F48BC280918C0392
:102BD000811509F4B9C3C0901B04D0901A040E9457
:102BE000660788579C4E90938E0380938D03D70180
:102BF00015968C91811509F4A7C38D2D8C298D799B
:102C000081115EC30115B0E51B0708F0E6C201158E
:102C1000E0E41E0708F081C3063E110509F40BC36A
:102C2000C80190528115904208F07EC3D7011696D4
:102C30008C91803108F43BC3C801992710921D0480
:102C40008D32910509F0E2C282E080931D0470C3C9
:102C5000003E42E5140750F4003652E5150708F02F
:102C600077CFC80192558034910551CF98012757ED
:102C70003C472530310508F04BCF0937BCE71B072F
:102C800009F04DC02091740330917503232B69F135
:102C9000811599F081E00E94AD0680916C03C4D942
:102CA00089E0EDE6F3E0A3E2B3E001900D928A95AE
:102CB000E1F7809177038093220386E0F701A3E296
:102CC000B3E001900D928A95E1F780912203809301
:102CD000810383E293E0C5DE10928103F7018581D1
:102CE000811103C080916C03A8D980911E04877064
:102CF000811561F0D70115968C91811539F080917D
:102D0000D50482FF03C082E00E9471032A96E2E1AB
:102D10000C940D31D70116968C918031F8CE0A377C
:102D2000FCE71F0709F014CF811509F4C5C0A09076
:102D30007403B090750320916C032D832983BE0129
:102D40006F5F7F4FC5010E94BB052C0139813A8717
:102D5000BCE2CB2EB3E0DB2E01E010E022242A946B
:102D6000D60117963C90179733FE53C06D907C9018
:102D7000119712968D909C90139746145704B9F4AE
:102D80001496BC91B987232DF60146816B2F8A8555
:102D90000E94D505811559F089850E94AA0228163E
:102DA00034F4D60115969C918401192B282E4814D1
:102DB0005904C9F431FE17C0F601F581F987232DB6
:102DC000D60116964C916F2F8A850E94D5058115E4
:102DD00051F089850E94AA0228162CF4F6019481EC
:102DE0008301192B282E30FE14C0FFEF2F1211C0C3
:102DF0000130110571F4232DD60116964C9160E037
:102E00008A850E94D505811521F0F601858184010E
:102E1000182BF8E0CF0ED11C2CE633E02C153D0525
:102E200009F09ECF01301105E1F58D8182958F70FB
:102E30003D81832B8F7011E0303108F410E0129542
:102E4000107F182BA11440E2B40620F5A11451E024
:102E5000B50608F055C00A2D812F8D704A2D8115B9
:102E600009F451C06AE086EB94E00E94BE06282F68
:102E700030E02115310551F4402F6EE180E994E0F6
:102E80000E94BE06282F30E0811549F0F901F12B90
:102E90008F0107C0C50190528115904390F100E069
:102EA00010E087E0E8E7F3E0DF011D928A95E9F79B
:102EB0001093800300937F0380917F0390918003A0
:102EC000892B09F412CFF7018581811539F08FEF35
:102ED0000E94AD06809177038093760386E0F70128
:102EE000A8E7B3E001900D928A95E1F7809176030F
:102EF0008093810388E793E0B4DD10928103F5CEDF
:102F00001B29BB24A8CF68E08EEA94E0AECFC801AD
:102F100097578038910508F0EFC0003108F0E5CEF2
:102F200066E870E080E090E0E3DB8111DECE812C8A
:102F3000912C5401011144C004E0AE014F5F5F4F7A
:102F40006A01D601E02F1D92EA95E9F724013501C7
:102F5000FFEF4F1A5F0A6F0A7F0AC501B401C8DB91
:102F60008983811509F4C1CE813009F0ACC0A50177
:102F700094012E5F3F4F4F4F5F4F2D833E834F8312
:102F80005887C301B201B4DB182F8A83811509F475
:102F9000ACCE8FEF810F833058F56D817E818F81AC
:102FA0009885A6DB8B83811519F0C6010E94BF0F9F
:102FB0002401350133E0430E511C611C711C46C0D5
:102FC000F7E88F169104A104B10409F48ECEC5016F
:102FD000B4018EDB2FEF821A920AA20AB20A811183
:102FE000EFCF0150A7CF4D805E806F8078842EC0D8
:102FF0008BEF810F833098F52401350143E0440EB7
:10300000511C611C711C6D817E818F81988570DBE4
:103010008B838115D9F0C301B2016ADB8C838115E2
:1030200071F08B819C8181305FEF950710F0982FB4
:103030008827163071F0173079F00E94542524014A
:10304000350154E0450E511C611C711C53014201B5
:1030500078CF0E941225F3CF0E943325F0CF143091
:1030600009F0C1CF6D817E818F81988541DB182F5A
:103070002401350184E0480E511C611C711CC501FE
:10308000B4016D5F7F4F8F4F9F4F32DB111509F4F5
:103090002CCE811509F429CE8150990B4FEF489F12
:1030A0009001499F300D1124A12FA150BB0B2A0F75
:1030B0003B1F2150310950F2EFE9FFE03197F1F762
:1030C00000C00000F6CFC6010E94BF0FBFCF223064
:1030D00009F07CCD2091860330918703232B09F4DE
:1030E00075CDFC01EB56FC4F20812E7F208380574D
:1030F0009C4F0E944C106ACD03375CE71507B9F46A
:1031000080918C03811519F00E942710EECD10924A
:103110001B040E949A030E94660788579C4E909356
:103120008E0380938D0381E080938C03DECD023A81
:1031300082E51807C1F158F4C801905281159042F8
:1031400020F1013E110579F1053E110503C0023B56
:10315000B2E51B0709F03ACD25EE30E027703327A2
:1031600081E090E001C0880F2A95EAF720918F0353
:1031700030918C033115F9F0D70115963C9131153A
:10318000A9F0282B20938F03B0CDF70186818031E1
:1031900008F01CCD812F99278F71992782309105D6
:1031A00011F04297D7CF21EE30E0D8CF809582231F
:1031B00080938F039ACD322F3823311509F406CD31
:1031C000982F9095922390938F030E949203F7017A
:1031D0008581811509F489CDF9CC003EB2E51B0744
:1031E00008F058C0003CE2E51E0728F5003AF2E579
:1031F0001F07E8F4003622E51207E8F4C8019255EB
:1032000080349105C0F010921D04C8018E329105E2
:1032100008F0E1C08832910508F088C08E31910530
:1032200008F086C004974A9708F40ECD49C0043BC5
:1032300032E5130741F7D7011596DC90D11409F454
:10324000ACC117FFAAC12801E89457F8612C712C72
:103250000E94D8068093150490911604913029F4A9
:1032600081FF03C089E30E94460F80911B04809375
:10327000140410921B0410921D04809116048230D5
:1032800009F41BC108F0E0C0811110C182EE0E9458
:10329000740EE0C009374CE7140728F407375CE7E1
:1032A000150748F6B0CF0B378CE71807C3CF812F2F
:1032B0008F71843109F4BFCF863149F410921D0417
:1032C0000E94271080918F030E948C033DC00E94B2
:1032D000271080918F030E948C03F701858181154F
:1032E00009F4A9CF0533FCE71F0709F4A9C008F0CA
:1032F00096C003333CE7130709F49EC004334CE740
:10330000140709F49BC002335CE7150709F093CF5B
:10331000109216040E94FF0A8ECFD70116968C9148
:10332000803108F089CCD9CFC80188CC8A9741F682
:1033300080918F03811531F080911D0492E08927DF
:1033400080931D040E942C0BC80197558115914054
:1033500020F65801F8EFAF22BB24A114B10409F004
:10336000C4CCF801FF2774E0EE0FFF1F7A95E1F758
:103370009F0120573C4F6901D70115968C91EB5660
:10338000FC4F908180FB90F99083811559F10E9448
:1033900066079093130480931204F60182818F5F75
:1033A000828380911D0490911B04892B83838091DB
:1033B0001A0484834681578166857785C6010E94F9
:1033C000D306D60115968C9181FF5801B092110455
:1033D000A092100482CF8C34910509F4A9CF8D32CC
:1033E0009240A5CFF9014485558566857785C90149
:1033F0000E94D306D60115968C9181FF6ECFC6012F
:103400000E94301080911004909111040817190740
:1034100009F063CF10921104109210045ECF0633AE
:103420008CE7180779F085E007339CE7190709F066
:1034300002CF809316046ECF81E0FBCF82E0F9CFFC
:1034400083E0F7CF84E0F5CF843009F44AC08530BB
:1034500009F44CC08FE39CE90197F1F700C000002C
:10346000C09016045CE1852E912C67E0A62EB12C4D
:10347000D301C201082C04C0B695A79597958795EE
:103480000A94D2F7E82FEF703E2ED11451F0F4E0F9
:10349000CF12D2C42AE0E21708F4CEC480E00E9422
:1034A000A70F832D0E94A70FD12CCDC460E070E040
:1034B00088E193E00E94180FCDCF8091150480FD24
:1034C00003C083E50E94460F82EE0E94740EEFE374
:1034D000FCE93197F1F700C0000087E50E94460F34
:1034E000B9CF86EE0E94460F88E1F8CF60E070E029
:1034F0008BE191E00E94180F60E070E085E290E0BF
:103500000E94180F60E070E088E290E0D3CF843032
:10351000D9F18530D9F18091140480931B04D7012F
:1035200015969C91911509F4AAC41092170498015C
:1035300030572332310508F0B2C484E090E00E9495
:10354000AA319093D5048093D404F801E150F04758
:10355000E232F10508F058C0EE5EFD4C0C943B31B0
:103560008CE20E94460F8091150481FFD4CF89E33D
:103570000E94460FD0CF82EE0E94D40E8091150497
:1035800080FDC9CF83E5F4CF88E2F2CF60E070E040
:1035900088E290E00E94180FBECFF801E851FC4786
:1035A000E730F10508F0BBCFEC5CFD4C0C943B31EF
:1035B00006E221EE41EE6AE17CE78D2DF4D995CB50
:1035C00007E225EE45EE6BE17CE7F7CF06E221EE60
:1035D00040EE68E17CE7F1CF07E225EE44EE69E1D9
:1035E0007CE7EBCF06E221EE42EE6CE17CE7E5CF33
:1035F00007E225EE46EE6DE17CE7DFCF08E221E051
:1036000045EE6EE17CE7D9CF8091D4048160809350
:10361000D4046091D4047091D50484E090E00E94B9
:10362000D8310E94790B61CB8091D504886080935A
:10363000D504EFCF8091D4048260E9CF8091D40487
:103640008460E5CF8091D4048860E1CF8091D50477
:103650008160EDCF8091D5048260E9CF8091D40460
:103660008061D5CF8091D4048062D1CF8091D40481
:103670008064CDCF0E94790B8091D4048068C7CF3D
:103680008091D4048C60C3CF8091D5048360CFCF68
:103690008091D4048E7FBBCF8091D504877FC7CF24
:1036A0008091D4048D7FB3CF8091D4048B7FAFCF32
:1036B0008091D404877FABCF8091D5048E7FB7CF24
:1036C0008091D5048D7FB3CF8091D4048F7E9FCF1E
:1036D0008091D4048F7D9BCF8091D4048F7B97CF32
:1036E0000E94790B8091D4048F7791CF8091D4047C
:1036F000837F8DCF8091D5048C7F99CF8091D40426
:10370000992782FF939590FB82F990FB83F97FCFF5
:103710008091D504982F909590FB80F990FB81F9CA
:1037200086CF9091D404892F8F7B96FF80646FCFD2
:103730000E94790B9091D404892F97FB87F98058C8
:1037400066CF61E08EE090E00E94BE3162CF60E023
:10375000F9CF9091D404892F8F7E94FF806157CF49
:103760009091D404892F8E7F90FF816050CF9091EB
:10377000D504892F877F93FF886059CF0737BCE72F
:103780001B07F9F00837ECE71E0731F19801205EBE
:1037900032452032310528F5911123C00F7181E0A7
:1037A00090E09C0102C0220F331F0A95E2F78901C5
:1037B000622F83E090E00E94BE31802F0E94C00201
:1037C00094CA81E0911551F00E94C60243E062E084
:1037D00081E00E94480389CA82E0F4CF0E94D002AF
:1037E000F5CF409119048091D304282F30E0209523
:1037F000309570E024233723232B19F0482340937E
:1038000019040B373CE7130741F4911509F46DCA0D
:103810000E94AD020E94330668CA003442E51407D4
:1038200008F055C0003252E5150708F057C00115E1
:1038300080E5180750F50115A0E41A0708F064C0E8
:10384000911509F479C00A35FCE71F0709F4CDC0CA
:1038500008F0B2C001303CE7130709F4C4C00330DC
:103860004CE7140709F4B9C001151C4709F064C0FE
:103870000E94790BAFEFB4E3ECE0A150B040E04020
:10388000E1F700C000000E94A308980130552115FF
:103890003240B0F6980145E0369527954A95E1F714
:1038A000822F8F702091190430E041E050E0082E03
:1038B00002C0440F551F0A94E2F724233523232B1B
:1038C00009F4BECF9111A6CF10921B04FEC298013D
:1038D000205C32452032310508F0B2CF802F8F7145
:1038E0002091190430E041E050E0082E02C0440F5E
:1038F000551F0A94E2F724233523232B09F4A0CF84
:10390000911509F4F2C986CFF7018681803108F05C
:1039100097CF911111C0212F2F7081E090E002C04C
:10392000880F991F2A95E2F72091190430E082232D
:103930009323892B09F0D9C9F701878190850097D6
:1039400009F457C00E9498048C01F701B580A68045
:10395000A2942FE0A22280911E048770811501F1AC
:10396000CB2CB114F1F0812F807F803461F080E2A4
:10397000800F8830A8F0812F807E803221F40230C1
:1039800078F0A11469F08091D50482FF09C082E02B
:103990000E94710380911E048770CC24C39481110E
:1039A000C12CE12FE295EF70103C08F094C0F0E0DC
:1039B000E55CFD4C0C943B310B358CE71807B9F0F6
:1039C0008091D504002482FF0394802D0C351C4780
:1039D00009F0B2CF0E94E90AAFCF6FEF7FEF80E02E
:1039E00090E00E94D8310E949C0B81E0F3CF80E0F0
:1039F000F1CF8581C080D180811569F0C6010E9418
:103A0000ED12182F682FC6010E94DE02B601812F29
:103A10000E94D21297CFC6010E941403182FF6CF2E
:103A2000F12FFF70DF2E103118F0D29490EFD922D1
:103A3000B114A9F0D11459F080E2800F883010F051
:103A4000011107C08D2D0E948C030E942C0B802F2A
:103A500040C080911D048D2980931D04F6CF802FD6
:103A60000E94D40ED114B9F180E2800F883010F09A
:103A7000011104C08D2D0E94920306C0D094809144
:103A80001D048D2180931D040E942C0B24C0212F26
:103A90002F70D22E107F103219F0D29480EFD822DE
:103AA000011549F0013009F483C0B11409F48FC045
:103AB000A114A9F1CCCF8091D50482FD2CC0B11402
:103AC00021F1D11429F08D2D0E948C030E942C0B22
:103AD00080E00E94740EC11409F4D9C080911E04C4
:103AE00080FDD5C0D70115961C9286958695869542
:103AF0000E94C602C7010E94311580911E0486955E
:103B0000869586950E94D002C2C080E00E94D40EA5
:103B1000D11409F3AFCFB11469F1A11004C08D2DF8
:103B20000E940810D8CF31E0A31210C010911A04DF
:103B30008D2D8123D81679F20E9466079093220476
:103B4000809321041D2910931A04C5CF45E0A412C7
:103B5000C2CF8D2D0E9408108D2D0E948607809166
:103B60001C049D2D9823D91609F4B5CF8D29809377
:103B70001C04B1CFA11012C08D2D0E940E108D2DEE
:103B80000E94860780911C049D2D9823911509F4AD
:103B9000A2CFD094D822D0921C049DCF51E0A51280
:103BA0009ACF80911B048D21811509F494CFE4CF25
:103BB000B11429F086E0A81608F08DCFB0CF95E0BB
:103BC000A91608F088CF8D2D0E940E1084CFA11465
:103BD000D1F3093349F4AFEFB7EEE3E0A150B040C1
:103BE000E040E1F700C00000802F0E94D40E73CFA8
:103BF000812F869586958370811561F0813009F05B
:103C00006ACFC8019370B11002C080E090E00E94BA
:103C1000130761CFC8019370B11002C080E090E03B
:103C20000E94EB0658CF6B2D802F0E94C40753CF04
:103C3000812F8370811138C0B11027C0402F429569
:103C400046954770440F440F802F8F70042E01C09B
:103C5000880F0A94EAF7202F207104FF07C02FE095
:103C600030E001C0220F4A95EAF720951695169587
:103C700013701230A1F0133081F03091D204113062
:103C800059F0822B83230E94C0020E94D80660E074
:103C9000C7010E9417133AC8832B822BF4CF822BC3
:103CA0009091D2048927EFCFB11451F110FFEDCFDD
:103CB000402F429546954770440F440F802F8F70D8
:103CC000042E01C0880F0A94EAF7202F207104FF08
:103CD00007C02FE030E001C0220F4A95EAF7209597
:103CE000169516951370123089F0133069F03091E3
:103CF000D304113041F0822B83230E94C302C5CF2D
:103D0000823018F2D5CF832B822BF7CF822B909164
:103D1000D3048927F2CF1F70B11439F0812F0E948C
:103D2000C602802F0E940810B0CF802F0E940E1074
:103D3000812F0E94D002A9CF023F71F170F4003FA1
:103D4000C9F0013F91F0B11409F465C0A11409F460
:103D50005FC0802F0E94740E98CF033F21F1043F73
:103D600091F78091D50482FD2AC0812F8F71B11403
:103D700001F316C0B11469F0F5E0AF1608F085CF75
:103D80001F7181E090E0012E01C0880F0A94EAF7CC
:103D9000BECF26E0A216F2CF812F8F71B110C9CF0E
:103DA0000E94C60272CF80E0B11409F4A6CF1F7141
:103DB00081E0012E01C0880F0A94EAF79ECFB1146A
:103DC000C1F080911E048770843049F410921E0463
:103DD0001092200410921F04812F8F71AACF35E01A
:103DE00063E0A31608F051CF812F8F710E947207F4
:103DF0004CCF45E0A41640F010921E04109220040F
:103E000010921F0464E0F0CF81E00E9471033DCF67
:103E1000812F8F71C5CFA114F9F2093349F45FEFF7
:103E200087EE93E0515080409040E1F700C00000E1
:103E3000802F0E94D40E29CF311033CB34E0A3164B
:103E4000B1040CF42ECB41E0A41AB10854E0851A59
:103E500091088FEFA816B80609F00ACB80911604D6
:103E6000823009F488CB08F052CB811179CB82EEF5
:103E70000E94D40E50CB0337BCE71B07ABC90631F9
:103E8000FCE71F0709F07ACC8091180465E38111E3
:103E900001C069E28AED91E00E94550716C0063123
:103EA0002CE7120709F06ACC80911B048A7A91E012
:103EB000811101C090E09093180465E3811101C065
:103EC00069E28AED91E00E943B070E942C0B0C9462
:103ED0007516A0E0B0E0EFE6FFE10C94FC308091B5
:103EE0000703803108F049C080910603811509F469
:103EF00044C0C091B80289E0D82E8091B7028C17D7
:103F0000E1F1EC2EF12CDC9EE0011124FE01E754DE
:103F1000FD4F84818115B1F1918180910203981345
:103F200031C090818091010398132CC0858181114B
:103F300029C0028113818091030390910403081B1F
:103F4000190B60E081E093E00E9417130E94B814FF
:103F500008171907B8F4809107038F708061809368
:103F60000703C154DD4F88818F708061888381E0B1
:103F700093E00E9431150E946703CDB7DEB7E7E0FA
:103F80000C941831E7012196C770B7CFAFE0B0E0CD
:103F9000ECECFFE10C94F4308C0186E0F801DE01DA
:103FA0001A9601900D928A95E1F7F801F580E48068
:103FB00081E0882E83E0982E80910503811117C03F
:103FC000E11491F0F11409F480C1C8010E94461374
:103FD000811509F47AC189E0F801A1E0B3E001900C
:103FE0000D928A95E1F775DFFF24F3946AC0A280F1
:103FF000B380D090060380910303909104033501B0
:10400000681A790AD11409F411C1C080518060E0A6
:1040100081E093E00E9417130E94B8146816790695
:1040200008F0B6C0E11401F380910203F801918118
:10403000E0900703F0E1EF1608F064C0981320C089
:1040400090910103F801808198131AC02091080310
:1040500030910903878190852817390789F4F11079
:104060004BC08E2D8F7080618093070381E093E0B9
:104070000E94311580910703F8018683F12C21C03D
:10408000F1103AC040E0652D8C2D0E942E0A40E0D0
:10409000652D8C2D0E942E0AF82E8111EFCF8A8576
:1040A0009B850E943913292F22952F70903470F42C
:1040B0009F702230A0F09115B1F0F80196819031F7
:1040C00090F48F2D2F96EFE00C9410312A5F2F7013
:1040D000223068F0C8010E943115FD2CF2CF9115F5
:1040E00011F0811571F3805E883058F3F3CF803F73
:1040F00040F3815F8330F9CF809107038160809323
:104100000703BCCF98131EC090910103F801808172
:10411000981318C020910803309109038781908576
:104120002817390779F4F1100DC0E682C8010E9402
:10413000311589E0F801A1E0B3E001900D928A9574
:10414000E1F752CFC8010E944613811509F4BDC0A2
:10415000F11409F4BAC080910703803208F43BCF10
:1041600080910103909102039A838983BC82AB8280
:10417000809105038D831E82EF82809108039091C8
:10418000090399878887CE0101960E94311523CFB4
:10419000D0900703F0E1DF1650F481E093E00E9435
:1041A000311589E0F40111928A95E9F767CFE1149E
:1041B00009F41ACF90910203F801818198131AC073
:1041C000909101038081981315C0209108033091CC
:1041D0000903878190852817390761F4F1100AC017
:1041E000D682C8010E94311589E0F40111928A95A6
:1041F000E9F7FACEC8010E944613811509F465C09B
:10420000F11409F462C080910703803208F4E3CE10
:1042100080910103909102039A838983BC82AB82CF
:10422000809105038D831E82DF82A7CF60E081E04D
:1042300093E00E9417130E94B8146816790608F0DC
:10424000B0CFE11409F4D0CEF11409F43EC090913E
:104250000203F801818198132EC09091010380819F
:10426000981329C020910803309109038781908514
:104270002817390701F58091030390910403A81AC8
:10428000B90AF8ECAF16B10408F053CF80910703D8
:1042900080FD4FCF803108F44CCFF8018683982FF2
:1042A000907F903F09F442CF982F907F905F8F705E
:1042B000892B86833BCFC8010E94461381118BCE88
:1042C00080910703816080930703C8010E94311524
:1042D0008BCEA2E1B0E0EFE6F1E20C94FF300A876A
:1042E0001B872C873D874E875F87688B798B8A8BEE
:1042F000CE010A964BDE811128C02091B702309181
:10430000B80289E0FE013A96DE01119601900D9205
:104310008A95E1F78E858115C1F0822F90E0019694
:104320008770992738171906D9F099E0929FD00124
:104330001124A754BD4FFE01319601900D929A951C
:10434000E1F78093B7020E94670319E08091B802F9
:104350009091B702891312C06296E4E00C941B316D
:104360000E94790B1092B7021092B80289E0E1E046
:10437000F3E0DF011D928A95E9F7E7CF189FC001AE
:10438000112487549D4F02DE811531F38091B802CC
:1043900090E00196877099278093B802D7CFEF926B
:1043A000FF920F931F93CF93DF938091CF04E091FF
:1043B0000A02CDE0811130C0CDB7DEB7E6E00C9443
:1043C0001931D1E0DE0FD0930A02EE2EF12CCE9FF0
:1043D000F0011124E959FB4F84818115E1F08781B7
:1043E0009085892B21F481859285019651F4008175
:1043F0001181228133814481558166817781808555
:1044000068DFCE9DF001CF9DF00D1124E959FB4FDF
:10441000148210921D04ED2F8091CF04E81788F2CA
:104420001092CF0410920A02C7CFA4E0B0E0EBE1F3
:10443000F2E20C94F23020916604298397E0992EE1
:1044400001E010E02DE0322E34E0532E88248394D6
:10445000809165049981891307C0A1DF0E94F60548
:104460002496E1E10C940E319981892F90E09C8390
:104470008B83FC01EE0FFF1FE55AFB4F808191817A
:10448000989ED001999EB00D1124FD01ED5DFB4F6A
:10449000FA83E983248121115BC06090CF04E7E6B1
:1044A000F4E060E070E0712C661508F04FC0A38462
:1044B000B484A981BA81CD90DC902FEF3FEF412CDD
:1044C000442D50E07601E40CF11CE40CF11CD70102
:1044D000ED90FC90E114F10439F0AE14BF0409F042
:1044E000A90143949A01ECCF2F3F3207D1F1D801B3
:1044F00002C0AA0FBB1F2A95E2F77A2A9801042C62
:1045000002C0220F331F0A94E2F7A901415051095A
:104510007416150629F5369EF001379EF00D11240C
:10452000E959FB4F989ED001999EB00D1124AD5DC5
:10453000BB4F12962D913C9113973087278354825D
:10454000108211829287818715968C920E940706AD
:104550008B819C8101969A8389838370898378CF2C
:1045600014826F5F7F4F3D969FCF1092D1041092BF
:10457000D00410923D0180916504809366040E94EE
:10458000F6050DCFACE1B0E0E8ECF2E20C94F130CE
:104590004B8B5C8B6D8B7E8B8F8BB92E988FA92E5E
:1045A000911110921D04188A198A1A8A86E0FE0158
:1045B0007396DE011A9601900D928A95E1F75F8855
:1045C0008091D50482FF1FC00E94660720911F04BE
:1045D00030912004821B930B8838934138F08091EE
:1045E0001E0482FD03C082E00E9471030E946607E0
:1045F0002091210430912204821B930B883893412F
:1046000010F00E949A035114D9F05E86BF8661E0D3
:10461000CE010A960E94171361E0CE010A960E940D
:10462000171361E0CE010A960E9417134C018035E2
:104630006CE7960791F4A11419F181E080933D0194
:104640005E86BF860A851B852C853D85452D5B2DA5
:10465000688979898A893DDECDC081359C4721F4FE
:10466000A11471F082DFECCF82E588168CE7980602
:1046700039F4A11429F080913D018111F3CFDDCFF0
:1046800043E2E42E44E0F42E412C612C712CD7013E
:104690006D917C91CC24CA94DD24DA9480E0282F9B
:1046A00030E0FB01E80FF11DE80FF11D4081518161
:1046B0004115510539F08416950609F096018F5F72
:1046C0006901EDCF10E0BFEFCB16DB0609F44EC059
:1046D000F701448110913D01411110E0D701159679
:1046E0003C90159716969C911697A11409F405C154
:1046F000111509F402C1311017C021E030E00C2C73
:1047000001C0220F0A94EAF7922B16969C932091EF
:104710006304309164042233310530F422E330E045
:104720003093640420936304E1E0F0E002C0EE0FF4
:10473000FF1F8A95E2F7CF010197D70116962C91BA
:104740002817190699F4C090D004D090D104C11450
:10475000D10409F453C00E9466078C199D09C397C0
:1047600008F44CC081E0F701848311E0412ABFEFD7
:104770006B1A7B0AE7E0EE0EF11CF8E06F1671048D
:1047800009F085CFA11409F417C1411409F414C12B
:104790000E9466079093D1048093D0048091CF0447
:1047A000883040F591E0980F9093CF0499E0FE0196
:1047B0003A96DE01119601900D929A95E1F75D828D
:1047C000BE822DE0829FC001112489599B4F29E0B0
:1047D000FE013196DC0101900D922A95E1F72FEF51
:1047E0003FEFDC011A963C932E9319971C969C92EE
:1047F0008E921B976C96E2E10C940D312091660429
:1048000080916504922FE0E0F0E001E0281709F4C0
:1048100048C0422F50E0FA01EE0FFF1FE55AFB4F50
:104820002080318037E0329DF001339DF00D11245E
:10483000ED5DFB4F608171817C8F6B8FB0E030E06C
:10484000A0E0EB8DFC8DEA0FF11DEA0FF11DC08099
:10485000D180C114D104E1F0F7010190F081E02D85
:10486000FA8FE98F30E007C0E1E0C616D70609F0FD
:10487000E0E0BE2B3F5FE98DFA8DE30FF11DE30F02
:10488000F11D608171816115710571F7AF5FD9CF3D
:10489000B11581F13A17C8F4E1E0D7011496EC9311
:1048A000F70190936604EE15FF0509F45FCF90E0E1
:1048B000FC01EE0FFF1FE55AFB4F718260820196EB
:1048C000837099278093650451CF37E0329DF001C2
:1048D000339DF00D1124ED5DFB4F0483EE15FF05B4
:1048E000F9F2291302C09F5F93709A012F5F3F4F27
:1048F00023708CCFE0E0F0E0F8CF292F30E03110CA
:1049000024C061E070E002C0660F771F8A95E2F76D
:10491000CB0101972817390791F010E0E1E0F0E0B2
:1049200002C0EE0FFF1FCA94E2F76F01C094D701D7
:1049300016968C9116978C2116968C9317CF41154D
:1049400069F3C3010E940706E8CFA9010C2C02C03D
:10495000559547950A94E2F7C9010197822393235D
:10496000892B39F540FF25C0D70112968D919C9176
:10497000892BD1F087E0FE013196DF011D928A95E7
:10498000E9F70E9466079C018B839C8384E08D83FA
:10499000F70192818381792F9887898709811A810C
:1049A00044E05E816F8195DCD70115961C92132D32
:1049B000B5CF142F1170B2CF909166048091650429
:1049C000981731F032DDB1E04B1609F413CF38CE31
:1049D000E6DC1092D1041092D0040E94F605F3CFC9
:1049E000A6E0B0E0E6EFF4E20C94FF300E94660728
:1049F0008C018091AB029091AC028017910771F00D
:104A000019821A820E946607BC0149815A8180E09E
:104A100090E0B8DD1093AC020093AB022696E4E080
:104A20000C941B31A6E0B0E0E8E1F5E20C94013112
:104A30009093A8028093A702811520E2920730F498
:104A40000E94BF0E2696E2E00C941D3180EF898310
:104A50008A830E9466078160BC0149815A8181E096
:104A600091E090DDEFCFA6E0B0E0E9E3F5E20C9451
:104A700001319093A8028093A702811520E292074A
:104A800030F40E94030F2696E2E00C941D3180EF73
:104A900089838A830E9466078160BC0149815A81AB
:104AA00081E090E06FDDEFCFCF93DF93D82FC92F58
:104AB000B9DF8D2F9C2FD7DFDF91CF9108950F9312
:104AC0001F93CF93DF938C01862F62E873E00E94DF
:104AD000A314892B91F4C0918203D0918303209772
:104AE00061F0F8018281833039F4CE01DDDFCE013F
:104AF000DBDFCE01D9DF01C0E0F7DF91CF911F915D
:104B00000F9108950F931F93CF93DF938C01EB01C7
:104B100062E873E08C2F0E94A314892B09F057C020
:104B2000FE01FF27D80112968C911297E55AFD4F8E
:104B30008130A9F415968C9182FD4EC080FF4CC047
:104B400082E0808380918403909185030097B9F47B
:104B500080918203909183030097C9F110C0823045
:104B6000A1F515968C9182FD26C080FD0AC083E0D8
:104B7000808380918603909187030097F1F052DF44
:104B800026C084E0808380918803909189030097F8
:104B9000B1F78091820390918303009701F184DF44
:104BA0008091840390918503009749F78091820357
:104BB00090918303E4CF85E080838091820390917C
:104BC0008303009721F070DFF1CF86E08083DF91CF
:104BD000CF911F910F91089581E08083B9CF80918B
:104BE000840390918503B8CF0F931F93CF93DF93E6
:104BF0008C01EB0162E873E08C2F0E94A314892BD7
:104C000071F4DD27C55ADD4F8881F80112821882C0
:104C10008330E9F048F4813059F0823081F0DF913F
:104C2000CF911F910F9108958430B1F08530B9F77D
:104C30008091820390918303009789F306C080914D
:104C4000840390918503009799F30DDFE8CF80915D
:104C5000860390918703F7CF809188039091890311
:104C6000009799F720918203309183038091840308
:104C70009091850321153105F9F2009731F7C901AB
:104C8000E4CFA0E1B0E0E7E4F6E20C94F330FE01FB
:104C9000319680E1DF011D928A95E9F709E010E085
:104CA00099E7A92E93E0B92E27E8422E512C612CCA
:104CB000712C4F0173016201B1E14B165104610483
:104CC00071041CF080E1C82ED12CA601B501C401ED
:104CD0000E94AF31AC0CBD1C0D2C000CEE08FF087F
:104CE0004C185D086E087F080150104019F7609657
:104CF000E0E10C940F316FEF85E290E00E94BE314D
:104D00006FEF86E290E00E94BE316FEF87E290E0A5
:104D10000E94BE3160E088E290E00E94BE310E94B5
:104D2000A113AFDF6DEB85E290E00E94BE316CE134
:104D300086E290E00E94BE3164EF87E290E00C943E
:104D4000BE31CDB7DEB7AC970FB6F894DEBF0FBE5D
:104D5000CDBF85B7806885BF85B7806885BF84B7BC
:104D6000877F84BF0FB6F894A89580916000886112
:104D700080936000109260000FBE80E890E00FB654
:104D8000F89480936100909361000FBE81E080935E
:104D9000030184E995E09093D9018093D8010E94A2
:104DA000A3050E941F140E9463140E945E090E94C2
:104DB000D4098091E20084608093E200789480912D
:104DC0008B02811599F08091E9001091EC008F70B1
:104DD000179511271795182B1092E9008091E8007C
:104DE00083FD0E94B10B1F701093E90082E084BD27
:104DF00093E095BD9AEF97BD80936E001092A30249
:104E00001092A4021092A5021092A6020E9488138A
:104E1000811101C070DF8091D80080618093D8003B
:104E20002AE12A95F1F700C08091D900182F11705E
:104E300080FD04C00E945E0910928B021093A102B3
:104E40001093A2021093180111110E949E2F8091BD
:104E50001801811112C084E1EEE3F1E0DE01119648
:104E600001900D928A95E1F784E1FE013196A4E06C
:104E7000B1E001900D928A95E1F78091180191E0DF
:104E80008927880F880F80936C0294E0981B909379
:104E90006B0224E031E061E070E0D90140E050E0D5
:104EA0008D918F3FA1F0E82FE295EF70F0E011A116
:104EB0008F707B0102C0EE0CFF1C8A95E2F7C701E0
:104EC0009E2D9095912391A392A1892B82A34F5F50
:104ED0005F4F4530510521F72B5F3F4F81E028316F
:104EE0003807D9F688E0E1E8F2E0DF01E82E1D920C
:104EF000EA94E9F7E3E6F2E0DF011D928A95E9F72B
:104F000080E090E00E94AA31833E9E4F21F40E94EF
:104F1000881381112DC063EE7EEF80E090E00E9447
:104F2000D83160E082E090E00E94BE3181E0809361
:104F3000D20461E083E090E00E94BE3160E074E161
:104F400084E090E00E94D83160E08CE090E00E9424
:104F5000BE31D1DE40E050E0BA018FE090E00E9427
:104F6000D03140E050E0BA0183E190E00E94D031BE
:104F700082E090E00E94A23180936F0284E090E092
:104F80000E94AA319093D5048093D4040E9471109A
:104F9000EFEFF6E721E0E150F0402040E1F700C0FC
:104FA00000000E9471108091A20291E08927880F71
:104FB000880FE82FF0E0EF57FD4F208130E041E00F
:104FC00050E0BA0102C0660F771F8A95E2F7CB0165
:104FD00082239323892B41F06FEF7FEF80E090E0F5
:104FE0000E94D8310E94A30883E090E00E94A23181
:104FF0000E94C0028CE090E00E94A23180931604CF
:105000008091A102811101C09CD789E191E0909328
:10501000AE028093AD0280918B02853049F480917D
:105020008B02853009F450C00E94790B0E94D8068B
:105030000E94711000E712E051E8E52E52E0F52ED3
:10504000D701F80191918D9168E772E06E177F07A3
:1050500009F471C09817B1F38090A102D12CD70147
:10506000CD907D01F80191908F019C1431F19C2429
:10507000B12CAA24A394892D8A218115B9F0811419
:10508000A9F0B982DA820E9466079C838B83F1E0E3
:10509000FD8391E08C2D8A21811101C090E09E83D7
:1050A00049815A816B817C818D816CDAB394AA0C21
:1050B00025E0B212E0CFF801C292D39438E0D312C7
:1050C000CECF0E948B083AC080918B02843021F1B0
:1050D00010926D0288E190E0A0E40FB6F894A895D4
:1050E000809360000FBEA093600083B7817F8460CF
:1050F00083BF83B7816083BF7894889583B78E7FA1
:1051000083BF0FB6F894A895809160008861809362
:105110006000109260000FBE0E947110E1E8F2E0A2
:10512000819181111CC579E8E72E72E0F72EEE1609
:10513000FF06B1F774CF98138FCF52DC8091A10294
:10514000811509F465C0E0901004F0901104E11499
:10515000F10439F1C0901204D09013040E94660744
:105160008C010C191D09C7010E94B8148017910702
:10517000C0F42091100430911104C9019927287FAF
:105180003327232B09F05BC144E0880F991F4A9510
:10519000E1F780579C4FDC0115962C9122FF0E946D
:1051A0004C1080913D01811511F10091D0041091B6
:1051B000D10401151105D9F00E946607801B910BDF
:1051C00020916304309164042817390780F490918A
:1051D000660480916504981709F434C126D91092A9
:1051E0006404109263041092D1041092D004809150
:1051F0008C03811569F00E94660720918D03309120
:105200008E03821B930B8F3F9F4710F40E94271041
:1052100086E0ECE1F3E0DE01119601900D928A95B3
:10522000E1F7B0901D0310911E03D0901F03C090B2
:1052300020030091210310921E0310921F0310926D
:10524000200310922103812F8D29811509F441C07B
:10525000E0907A02F0907B020E9466079C012E1972
:105260003F0990911A03911509F474C42531310551
:1052700080F19F3F19F09F5F90931A03111559F029
:105280000E94680691E011160CF09FEF899F802D17
:10529000112480931E03D11459F00E94680691E0F6
:1052A0001D140CF09FEF899F802D112480931F0304
:1052B00080911E03811569F0F0901F03F11449F0ED
:1052C0000E945A0680931E038F2D0E945A068093D7
:1052D0001F038C2D802B811509F441C0E0907802CA
:1052E000F09079020E9466079C012E193F09909167
:1052F0001903911509F429C42135310580F19F3F27
:1053000019F09F5F90931903C11459F00E94880609
:1053100091E01C140CF09FEF899F802D1124809345
:105320002003011559F00E94880691E010160CF038
:105330009FEF899F802D112480932103809120036A
:10534000811569F0F0902103F11449F00E945A068A
:10535000809320038F2D0E945A0680932103809111
:105360001D03B81219C080911E03811511F081131D
:1053700013C020911F03211511F02D110DC0909124
:105380002103911511F0901307C0309120033111C2
:1053900003C0822B892B81110E949B0786E0FE01AE
:1053A0003196ACE1B3E001900D928A95E1F70E944D
:1053B000D80690917C02891721F080937C020E948C
:1053C0007F0880918B02843009F025CE83E08093A2
:1053D000E9008091E80082FF1ECE8091E80090E015
:1053E00085FF0BC00E942D0930E2E32EF12C8E01C7
:1053F0000F5F1F4F8115C1F191E08091E8008B771D
:105400008093E800911509F406CE0091A90210914D
:10541000AA02E98101151105A9F1EE3F09F054C076
:105420008A81833020F08550833008F04DC0EA81B6
:10543000EE3008F049C0F0E0E95BFD4C1CC780E0AD
:1054400090E0A9CE0E94CF211092D1041092D004F6
:105450000E94F605CCCE8091F100F80181938F0176
:10546000F1E0EF1AF10841F28091E80085FDF3CFF9
:105470008091E8008B778093E8000E942D098115C8
:1054800099F3BACFE43148F4E11549F0E150E33142
:1054900030F4F0E0EB5AFD4CEEC6EE3F41F28FEFF8
:1054A000898312C01A8289E08B830EC08A81823080
:1054B00081F08330B1F0813091F70E947F08F1D6FE
:1054C0006B837C838D839E83CE0101960E947D0930
:1054D000A2CD88E290E036D71B821C821D828E838B
:1054E000F3CF8091890290918A02892B69F388E039
:1054F000E1E8F2E0DE01139601900D928A95E1F762
:10550000E3CF8A81823059F66B817C818D819E81C7
:10551000C8D688E290E032D7D7CF4C816B818A81A0
:105520000E94A3129827892798279E838D83CCCF2A
:105530002D813E813227232732274C816B818A813E
:105540000E94050BC1CF0E94A113BECF80E18A83C8
:10555000BBCF1A8287E8A8CF8C818D3108F0B4CFF9
:105560008A809B80982489249824A12CB12C9E01A8
:105570002F5F3F4F79018901080F111DE016F106D9
:1055800009F4A2CF80E037E883169104A104B104A6
:1055900020F4C40187589C4FD5D6D70114968C931C
:1055A000BFEFEB1AFB0AEFEF8E1A9E0AAE0ABE0A95
:1055B000E5CF8091890290918A02892B09F484CFEA
:1055C0008C818D3108F080CF882E912CA12CB12CAC
:1055D000CA80DB80DC24CD24DC24E12CF12C8E017C
:1055E0000F5F1F4F412C512C3201481459046A049B
:1055F0007B0408F069CFF7E8CF16D104E104F10489
:1056000038F4D80114966C91C60187589C4FB6D6D1
:10561000BFEF4B1A5B0A6B0A7B0AEFEFCE1ADE0A6A
:10562000EE0AFE0A0F5F1F4FE0CF2BDB4DCF88E065
:105630008ECF8C818D3108F047CF882E912CA12CF4
:10564000B12CCA80DB80DC24CD24DC24E12CF12CBD
:10565000412C512C32018E010B5F1F4F481459040D
:105660006A047B0408F030CF80E0F0E8CF16F2E067
:10567000DF06E104F10418F4C601899663D6D80167
:105680008D938D01BFEF4B1A5B0A6B0A7B0AEFEF1C
:10569000CE1ADE0AEE0AFE0AE1CF2C81022F10E0BC
:1056A0002D3108F011CF8A819B819827892798276F
:1056B0002C01612C712C8038F2E09F0708F004CF98
:1056C000822E912CA12CB12C40E852E060E070E0D9
:1056D0004419550966097709421751056105710595
:1056E00008F4F2CE2091890230918A02232B09F02E
:1056F0003EC01C0129E2220E311C80FBEE24FF2457
:10570000E0F880FF0BC088961DD69D8189279827D9
:10571000892781159C4711F48FEF8D83D501C40132
:10572000840D951DA61DB71D80FF19C0680161E09D
:10573000C61AD108CE0105968C0D9D1D9CA78BA77E
:10574000C101800F911FFED5ABA5BCA59C91811511
:105750009C4721F48FEFEBA5FCA580838601FE0119
:105760003196EE0DFF1D2FEFE016F10638F08E0199
:105770000F5F1F4FC12CD12C760125C094818581EC
:1057800081159C4711F42483258362E0E60EF11C09
:105790003296EACF70E8471672E05706610471044A
:1057A00030F4D80114966C91C2018996E7D5BFEF09
:1057B000CB1ADB0AEB0AFB0AEFEF4E1A5E0A6E0AFF
:1057C0007E0A0F5F1F4FC814D904EA04FB0410F3CC
:1057D0007BCE8091890290918A02892B09F474CE44
:1057E000CE0101960E947D09FFEF21EE34E0F150D9
:1057F00020403040E1F700C00000F4CB88E0E2E553
:10580000F1E0DE01919601900D928A95E1F7FE019B
:1058100032968FE1DF011D928A95E9F786E0898350
:1058200088E07F96DE01159667CE8CE3898381E060
:105830008A831B821C8248CE8B819C81092E000C9E
:10584000AA0BBB0B25E0880F991FAA1FBB1F2A9527
:10585000D1F7AC01BD01405E5F4F6F4F7F4F4817DE
:1058600059076A077B0708F42FCE8C33E1E09E07C7
:10587000A105B10508F028CE4D33F1E05F076105C1
:10588000710520F04CE351E060E070E0481B590BDB
:10589000BC016C5A7C4FCE0101961ED515CE4AE153
:1058A00050E06FEF70E0CE01079635D58091890208
:1058B00089830A831B821C8282E08D8383E00FCE62
:1058C00081E090E09093AA028093A90282E390E0A5
:1058D0009093800280937F020E94660790937E02DD
:1058E00080937D02F1CD0115110581F1D0908102E7
:1058F000C0908302E0907D02F0907E020E946607D5
:105900008E199F098536910540F1C3FE26C0D0FE51
:1059100024C00E94660790937E0280937D0280914E
:105920007F029091800201979093800280937F0282
:10593000892B61F41092AA021092A90281E090E0F2
:1059400090938A028093890200E010E0809189029E
:1059500089830A8380917F02A7CD82E390E09093B0
:10596000800280937F02F2CF10928A021092890205
:10597000ABCD40E250E06FEF70E0CE010196CBD4AA
:10598000A3CDEB81E93008F09FCDF0E0E859FD4C64
:1059900072C4FE0133968DE1DF011D928A95E9F70D
:1059A00088E089838A838C8383E088A38DCD8C8172
:1059B0009AE0F92E8E010F5D1F4FF801EF2C119226
:1059C000EA94E9F7B8010E94A3148983F801DE0183
:1059D000129601900D92FA94E1F776CD1C818AE03F
:1059E000FE013596DE01919601900D928A95E1F7C0
:1059F00089A19AA10E9496059AA389A38BA19CA133
:105A00000E9496059CA38BA38DA19EA10E94960542
:105A10009EA38DA38FA198A50E94960598A78FA3FA
:105A20008FEF183060F42AE0129FB00111246755FF
:105A30007D4F4AE050E0CE018196BED480E089835C
:105A40000E94A30541CD2C816AE0CE018196DC0144
:105A5000E62F1D92EA95E9F7283080F4629FB001A5
:105A6000112467507D4F4AE050E05CD480E0898388
:105A70008AE0FE01B196DE0112963ECD8FEFF7CFA0
:105A80001C818AE0FE013596DE01919601900D920F
:105A90008A95E1F789A59AA50E9496059AA789A7F4
:105AA0008FEF183060F4FAE01F9FB00111246750A7
:105AB0007D4F4AE050E0CE0181967ED480E089831C
:105AC0000E941F1401CD2C8166E0CE018196DC017D
:105AD000E62F1D92EA95E9F7283060F4629FB00145
:105AE0001124675B7C4F46E050E01CD480E0898342
:105AF00086E0BFCF8FEFFBCF1C8186E0FE0135969D
:105B0000DE01919601900D928A95E1F789A19AA103
:105B10000E9496059AA389A38BA19CA10E94960539
:105B20009CA38BA38FEF183060F4F6E01F9FB001A9
:105B30001124675B7C4F46E050E0CE0181963CD457
:105B400080E089830E946314BFCC2B30310508F0BC
:105B5000D8CB05CC2B30310508F08DCBBACB80915A
:105B60006E02811509F45BCA60E1F62EF9BC22E1F0
:105B700029BD09B400FEFDCF8091D8008F7D8093B0
:105B8000D8008091E00082608093E0008091E00086
:105B900081FDFCCF0E94790B42CA1F921FB61F9253
:105BA00011248F939F93AF93BF9380916D028111C6
:105BB00013C08091020290910302A0910402B0915F
:105BC00005024196A11DB11D80930202909303022C
:105BD000A0930402B0930502BF91AF919F918F9162
:105BE0001F901FBE1F90189578941F921FB61F928A
:105BF00011248F939F93AF93BF9380910202909152
:105C00000302A0910402B09105020196A11DB11DED
:105C10008093020290930302A0930402B0930502C2
:105C2000BF91AF919F918F911F901FBE1F901895AC
:105C30001F920F920FB60F9211242F933F934F9301
:105C40005F936F937F938F939F93AF93BF93EF93E4
:105C5000FF938091E10082FF09C08091E20082FF02
:105C600005C08091E1008B7F8093E1008091DA0094
:105C700080FF24C08091D80080FF20C08091DA008E
:105C80008E7F8093DA008091D90080FFA9C080E1E7
:105C900089BD82E189BD09B400FEFDCF81E080931A
:105CA0008B028091F101811109C00E945E090E945E
:105CB000D4098091E20084608093E2008091E10049
:105CC00080FF1AC08091E20080FF16C08091E20040
:105CD0008E7F8093E2008091E20080618093E200F9
:105CE0008091D80080628093D80019BC85E08093B1
:105CF0008B0283E0809303018091E10084FF2FC039
:105D00008091E20084FF2BC080E189BD82E189BDE2
:105D100009B400FEFDCF8091D8008F7D8093D8001C
:105D20008091E1008F7E8093E1008091E2008F7E80
:105D30008093E2008091E20081608093E200809194
:105D4000F001811509F452C084E080938B028091A8
:105D50008B02843009F052C082E08093030180916D
:105D6000E10083FF2CC08091E20083FF28C0809176
:105D7000E100877F8093E10082E080938B021092A4
:105D8000F0018091E1008E7F8093E1008091E2003C
:105D90008E7F8093E2008091E20080618093E20038
:105DA00042E060E080E00E94A4098091F0008860F9
:105DB0008093F00081E08093030180930201FF91C2
:105DC000EF91BF91AF919F918F917F916F915F9173
:105DD0004F913F912F910F900FBE0F901F901895EC
:105DE00019BC10928B021092F10168CF8091E300F0
:105DF00087FF02C083E0A9CF81E0A7CF81E0ADCFCC
:105E00001F920F920FB60F921124EF92FF920F93F1
:105E10001F932F933F934F935F936F937F938F9332
:105E20009F93AF93BF93CF93EF93FF9309EE10E04F
:105E3000F8018081C091EC008F70C795CC27C79581
:105E4000C82B108280EFE82EF12CF7018081877F2C
:105E5000808378940E94B10BF8011082F701808151
:105E600088608083CF70F801C083FF91EF91CF915C
:105E7000BF91AF919F918F917F916F915F914F9162
:105E80003F912F911F910F91FF90EF900F900FBEB8
:105E90000F901F9018958EE1489B02C08A95E1F7FC
:105EA000489BFECF0895589880E28A95F1F7589A5A
:105EB0000895FC012BE02A95F1F728E090E080E0BE
:105EC00031E040E14A95F1F7880F489B02C08160BC
:105ED000932742E04A95F1F7000040E14A95F1F737
:105EE0002A9579F720E12A95F1F729B132E03A9520
:105EF000F1F7000040E14A95F1F7217092272081E7
:105F0000920F90830895A1E0B0E0E8E8FFE275C148
:105F100019828C017C01E60EF11CBDDFCE010196D9
:105F2000C8DFF80181938F01EE15FF05B1F781E01D
:105F30009981911180E02196E6E07BC1509A589AB0
:105F400008955098589AE89AE9E6F0E080818C7FAD
:105F5000808308956150770B91E001C0990F6A9595
:105F6000EAF7692F90E021E0611108C0911599F0DE
:105F7000589A80E28A95F1F758980895362F382379
:105F8000311539F0589A922730E23A95F1F7669533
:105F9000EBCF5898F9CF5898ECCFFF920F931F93FF
:105FA000CF93DF93EC018C01060F111DF9907BDF7D
:105FB00068E08F2DCFDFC017D107C1F7CDB7DEB7AF
:105FC000E5E038C11F920F920FB60F9211240F9384
:105FD0001F932F933F934F935F936F937F938F9371
:105FE0009F93AF93BF93EF93FF93CF93DF930F9262
:105FF000CDB7DEB719824FDFCE0101965ADF082FE9
:10600000069506950695982F92959570202F2570E8
:10601000920F292F237096959695920F9827977037
:106020008981892B811509F058C0043008F055C0CA
:1060300080E18A95F1F7589A509A82E08A95F1F7B3
:1060400000C0589888E0089F80011124D801AB5DFA
:10605000BE4F1696ED91FC9117973097A9F060917D
:106060006A0170916B0114962D913C911597260F42
:10607000371F11968D919C911297680F791F139677
:106080004C9113978C910995F801EB5DFE4F63815C
:10609000611549F020916A0130916B0184819581ED
:1060A000820F931F7ADFFFDE80E18A95F1F758981F
:1060B0005098589A80E18A95F1F7F801EB5DFE4F10
:1060C0006081611549F020916A0130916B018181F5
:1060D0009281820F931F17DFDEDE0F90DF91CF9149
:1060E000FF91EF91BF91AF919F918F917F916F91B0
:1060F0005F914F913F912F911F910F910F900FBE84
:106100000F901F9018950F931F93CF93DF938C01DF
:1061100004970CF05EC0F894509A589885E08A95E0
:10612000F1F70000C02FC695C570802F8570C80F8D
:106130008C2F8370C695C69593E0000F111F9A951A
:10614000E1F7C80FC8018C2BEC01ADDE00C068E0A0
:106150008C2F00DF90E19A95F1F75098589A489B60
:1061600031C087E090E048992FC0F801EB5DFE4F09
:106170006381611559F020916A0130916B0184812E
:106180009581820F931FBFDE811501F184DE80E2CD
:106190008A95F1F75898509A90E19A95F1F7F8019D
:1061A000EB5DFE4F6081611549F020916A013091ED
:1061B0006B0181819281820F931FEFDE74DE7894F0
:1061C00081E008C000C0CBCF019749F4509A589A9B
:1061D000789480E0DF91CF911F910F91089500C0D6
:1061E000C2CF2F923F924F925F926F927F928F9287
:1061F0009F92AF92BF92CF92DF92EF92FF920F9356
:106200001F93CF93DF93CDB7DEB7CA1BDB0B0FB65F
:10621000F894DEBF0FBECDBF09942A88398848881C
:106220005F846E847D848C849B84AA84B984C884B2
:10623000DF80EE80FD800C811B81AA81B981CE0FA9
:10624000D11D0FB6F894DEBF0FBECDBFED0108958E
:1062500097FB072E16F4009406D077FD08D028D0BF
:1062600007FC05D03EF4909581959F4F0895709559
:1062700061957F4F0895EE0FFF1F0590F491E02D7B
:106280000994082E817006940694811D0694811D40
:106290000694811D0694811D0694811D0694801D1F
:1062A00008956927962769277827872778270895EB
:1062B000AA1BBB1B51E107C0AA1FBB1FA617B7072C
:1062C00010F0A61BB70B881F991F5A95A9F7809548
:1062D0009095BC01CD010895FB01DC0102C0059041
:1062E0000D9241505040D8F70895FB01DC0104C0E5
:1062F0008D910190801921F441505040C8F7881BBE
:10630000990B0895FB01DC0102C001900D924150F0
:106310005040D8F70895DC0101C06D9341505040C2
:10632000E0F70895DC01CB01FC01F999FECF06C02E
:10633000F2BDE1BDF89A319600B40D924150504043
:10634000B8F70895F999FECF92BD81BDF89A9927C3
:1063500080B50895A8E1B0E042E050E0E5CFDC016F
:10636000A40FB51F4150504040F0CB01840F951F42
:106370002E9105D041505040D8F70895262FF99915
:10638000FECF92BD81BDF89A019700B4021639F094
:106390001FBA20BD0FB6F894FA9AF99A0FBE089565
:1063A0000396272FECDFEADF252FE9DF242FE7CF45
:1063B0000196272FE4DFE2CFDC01CB0102C02D9153
:1063C00005D041505040D8F70895262FF999FECFB7
:1063D0001FBA92BD81BD20BD0FB6F894FA9AF99A02
:1063E0000FBE01960895F894FFCFD007D507D707C1
:1063F000DC07EC07EC07EC07EC07EC07EC07EC0715
:10640000EC07DE07E207E507EA07FA0700080408D9
:106410008E0CB40CBA0CB40CBA0C0C0D2D0DBA0CBD
:10642000330E400E481BB01B501B1A1B1E1B541B67
:10643000221B581B641B2E1BA91B321B681B361BFF
:106440006C1B911B3A1B701B981B401B761B7E1B01
:10645000261B5C1B2A1B601B441B7A1B881BA11B71
:10646000A71B141B4C1BB71BE61AEC1AD81AE01A10
:10647000F21AF81AFE1A101D101D471D471DF81DAF
:10648000131E6B1D6B1D181E8B1E9C1E9C1EFE2B4F
:10649000152C1C2C642A642A4F2C602C732CB42CD1
:1064A000B92C642A642A642AC12C522A562A812AC9
:1064B0008D2A982AA32A4F2A4F2A4F2A4F2AE92B9E
:1064C000A62AA92AAC2AD92A152B172B192B4D2B12
:1064D000C92CD72CEE2C232D402D642A642A632D41
:0264E0007C2D11
:1064E20000000100F6359793FFF7F534669231F418
:1064F200C69491333236FFFF0163078F0AB408A5B1
:106502000AAA0A860A00000001000000000000003A
:106512000401000000040500000000000001939740
:1065220035F6FF926634F5F79194C6F4313632337C
:10653200FFFF195419979AE3F1ED0044227B4901B8
:106542002701AC004F02680288029002E200E900D3
:10655200EA00B500B600B700CD008301CC008A0185
:10656200920194012102230224022502260227021B
:106572002A02B300B4006F0070009F01CB019F029A
:10658200A002E200E900EA00B500B600B700CD00C3
:106592008301CC008A019201940121022302240288
:1065A2002502260227022A02B300B4006F007000FF
:0865B2009F01CB019F02A00232
:00000001FF
